S01E00002E2E5C62696E5C6F70656E626C745F786D63343730302E7372656353
S3150800000000600020191200085F120008611200083B
S315080000106312000865120008671200080000000055
S31508000020000000000000000000000000691200083F
S315080000306B120008000000006D1200086F1200081D
S315080000407312000875120008771200087912000862
S315080000507B1200087D1200087F1200088112000832
S3150800006083120008000000000000000000000000E5
S31508000070851200080000000087120008891200088F
S315080000808B1200088D1200088F12000891120008C2
S315080000909312000895120008971200089912000892
S315080000A09B1200089D1200089F120008A112000862
S315080000B0A3120008A5120008A7120008A912000832
S315080000C0AB120008AD120008AF120008B112000802
S315080000D0B3120008B5120008B7120008B9120008D2
S315080000E0BB120008BD120008BF120008C1120008A2
S315080000F0C3120008C5120008C7120008C912000872
S31508000100CB120008CD120008CF120008D112000841
S31508000110D3120008D5120008D7120008D912000811
S31508000120DB120008DD120008DF120008E1120008E1
S31508000130E3120008E5120008E7120008E9120008B1
S31508000140EB120008ED120008EF120008F112000881
S31508000150F3120008F5120008F7120008F912000851
S315080001600000000000000000000000000000000081
S31508000170FB120008FD120008FF1200080113000810
S3150800018003130008051300080713000809130008DD
S315080001900B1300080D1300080F13000811130008AD
S315080001A0131300081513000817130008191300087D
S315080001B01B1300081D1300081F130008211300084D
S315080001C0231300082513000827130008291300081D
S315080001D02B1300082D1300082F1300080000000039
S315080001E031130008331300083513000837130008C5
S315080001F039130008000000003B1300080000000047
S3150800020010B5054C237833B9044B13B10448AFF342
S3150800021000800123237010BD80000020000000002C
S31508000220981C0008084B10B51BB108490848AFF3DD
S3150800023000800848036803B910BD074B002BFBD0A4
S31508000240BDE81040184700BF0000000084000020E9
S31508000250981C00086C00002000000000154B002BBD
S3150800026008BF134B9D46A3F5803A00218B460F46DF
S315080002701348144A121A01F053FC0F4B002B00D0F6
S3150800028098470E4B002B00D0984700200021040009
S315080002900D000D48002802D00C48AFF3008001F08D
S315080002A019FC2000290000F06BFD01F0FFFB00BFE0
S315080002B000000800006000200000000000000000A8
S315080002C080000020940900200000000000000000C3
S315080002D008B500F045F8044B5B6A13F4005F01D1DA
S315080002E0002008BD012008BD008F024808B564201B
S315080002F000F006F808BD00BF08B500F007F808BD0D
S31508000300014B1880704700BFA000002008B501F017
S315080003105FF80F4B1B68984218D30E4B1B783BB9F6
S3150800032001220C4B1A704FF400720B4B5A6006E010
S315080003300022084B1A704FF00072074B5A6001F002
S3150800034047F8064B1B881844014B186008BD00BFC8
S315080003509C000020A200002000850248A000002082
S315080003604FF00072014B5A60704700BF0085024883
S3150800037082B00023019303E000BF019B0133019380
S31508000380019B8342F8D302B0704700BF72B60D4B8B
S315080003900D4A9A60BFF34F8F62B6D3F8882042F4AD
S315080003A07002C3F888205A6922F008025A61074980
S315080003B041F214028B5823F00F0343F004038B50C9
S315080003C0704700BF00ED00E000000008001000586C
S315080003D000487047001BB70010B51E4BDB6813F4C6
S315080003E0803F27D01C4BDB6813F0010F02D1FFF7C3
S315080003F0EFFF00E01948184B1B6813F0040F11D0E3
S3150800040015498A68C2F303628B68C3F306238C68AE
S31508000410C4F30644611C02FB0112B0FBF2F203FBB3
S31508000420022208E00C4B9B6803F07F030133B0FB04
S31508000430F3F200E0094A0749C868C0B20130B2FBC6
S31508000440F0F3086900F001000130B3FBF0F0044B4B
S31508000450186010BD004600501047005000366E0167
S315080004606C00002070B5574B1B6813F0010F09D1BB
S31508000470544A536843F001035360524B1B6813F008
S31508000480010FFAD0504B1B6813F4007F08D04E4A70
S31508000490936843F40073936041F64C50FFF768FF86
S315080004A04A4C636843F40023636040F6C410FFF7C0
S315080004B05FFF636823F4803323F002036360444BD1
S315080004C05B6813F0300F21D0103C636823F4702367
S315080004D023F030036360FFF77BFF3E4BA3FB00234B
S315080004E01B0D013B626842EA03436360374BDA68D7
S315080004F022F00102DA605A6822F400325A60334B5D
S315080005001B6803F46073B3F5607FF8D12F4B5A6804
S3150800051042F001025A605A6842F010025A602E4AA6
S315080005209A605A6842F040025A605A6822F01002ED
S315080005305A605A6842F480225A60244B1B6813F0AA
S31508000540040FFAD0214A536823F0010353601F4B66
S315080005501B6813F0010FFAD1204C4FF00113E3602A
S31508000560002666612661266266620323E3611C4BE8
S31508000570A3611C4BA362154D6B6823F040036B60A7
S31508000580194BAB604FF41660FFF7F2FE174BAB60E2
S315080005904FF46160FFF7ECFE154BAB604FF49650D5
S315080005A0FFF7E6FE134BAB6041F27070FFF7E0FE13
S315080005B0114BAB604FF4E150FFF7DAFE6660FFF7C8
S315080005C00BFF70BD00420050004400501047005019
S315080005D0004700506BCA5F6B002F0B0100460050A6
S315080005E00500010003002001002F0501002F03016B
S315080005F0002F0201002F0101002F000110B54FF056
S315080006000053044C0FCB84E80F00FFF7BFFEFFF73B
S3150800061029FF10BD700000205022014B1A60704758
S315080006205455000C024B186004331960704700BF1C
S31508000630F055000C10B4064AAA2313605524054940
S315080006400C60A021116003605DF8044B704700BF81
S315080006505455000CA8AA000C30B4074BAA241C60F9
S31508000660064A5521116080251D601C6011603023E3
S31508000670036030BC704700BF5455000CA8AA000C94
S31508000680F522014B1A6070475455000C41F21003CD
S31508000690014AD058704700BF0010005870B506468A
S315080006A00D46FFF7EDFFFFF7B7FF002407E0631CD1
S315080006B055F8231055F82400FFF7B4FF02343F2CF1
S315080006C0F5D93046FFF7B6FF41F21003024AD35870
S315080006D013F0010FF8D170BD0010005810B504468C
S315080006E0FFF7CEFF2046FFF7B7FF41F21003034A94
S315080006F0D35813F0010FF8D110BD00BF00100058F1
S31508000700F8B504460D461646624B98422FD003F5B7
S31508000710807398422BD003F58073984227D003F54F
S315080007208073984223D003F5807398421FD003F54F
S31508000730807398421BD003F58073984217D003F54F
S315080007408073984213D003F5807398420FD003F54F
S31508000750807398420BD003F5A063984207D003F53F
S315080007608073984203D043214B4800F00DFF33783D
S315080007701BB3082B23D0102B23D0182B23D0202BC8
S3150800078023D0282B23D0302B23D0382B23D0802BD3
S3150800079023D0882B23D0902B23D0982B23D0A02B83
S315080007A023D0C02B23D0C82B23D0D02B23D0D82B93
S315080007B023D0E02B23D1012322E0012320E00123CB
S315080007C01EE001231CE001231AE0012318E001239F
S315080007D016E0012314E0012312E0012310E00123AF
S315080007E00EE001230CE001230AE0012308E00123BF
S315080007F006E0012304E0012302E0012300E00023D0
S315080008001BB94421244800F0BFFEAB081F1D54F84D
S31508000810270005F00302D200F821914020EA0101E1
S3150800082044F82710606F6F000321B94020EA0101E0
S3150800083061671A498C4203D001F580718C4207D151
S31508000840216E012000FA05F521EA0505256617E05F
S315080008507168A9406160E908103154F8217005F003
S315080008600705AD000720A84027EA000044F8210044
S3150800087054F82170307A00FA05F53D4344F82150C2
S31508000880043354F82300317801FA02F2024344F89B
S315080008902320F8BD008002484C1B0008008E024841
S315080008A0030F20F0704003EB43039A00014BD0502E
S315080008B0704700BF14440050034B1868034B5B692C
S315080008C003F00103D84070476C0000200046005032
S315080008D0030F20F0704003EB43039A00014BD050FE
S315080008E0704700BF4846005070B504460E46154688
S315080008F0494B98422FD003F5807398422BD003F5C5
S315080009008073984227D003F58073984223D003F565
S31508000910807398421FD003F5807398421BD003F565
S315080009208073984217D003F58073984213D003F565
S31508000930807398420FD003F5807398420BD003F565
S31508000940A063984207D003F58073984203D04321E9
S31508000950324800F019FE1DB3082D23D0102D23D0E0
S31508000960182D23D0202D23D0282D23D0302D23D069
S31508000970382D23D0802D23D0882D23D0902D23D019
S31508000980982D23D0A02D23D0C02D23D0C82D23D019
S31508000990D02D23D0D82D23D0E02D23D1012322E03A
S315080009A0012320E001231EE001231CE001231AE0B5
S315080009B0012318E0012316E0012314E0012312E0C5
S315080009C0012310E001230EE001230CE001230AE0D5
S315080009D0012308E0012306E0012304E0012302E0E5
S315080009E0012300E000231BB944210C4800F0CCFD8C
S315080009F0B308043354F8231006F00306F600F82269
S31508000A00B24021EA020244F8232054F82320B540D4
S31508000A10154344F8235070BD008002486C1B00083B
S31508000A2070B505460E4600F0FDF8F47904B91024B1
S31508000A3022463168284600F047F8B379013B640836
S31508000A400134240244EA430343F4403343F00103E8
S31508000A50EB633379013B1B0643F481736B6373794C
S31508000A602BB16A6B013B42EA03436B6305E06A6B91
S31508000A703379013B42EA03436B634FF4A063AB63EC
S31508000A804FF0FF33EB6433892B6470BDD0F808311F
S31508000A9013F0E06F09D1836B13F0800FFBD14FF48D
S31508000AA00053C364C0F880107047C0F880117047BF
S31508000AB0D0F80C3113F0E06F02D1406D80B2704768
S31508000AC0D0F81C0180B2704763293BD9002A3BD075
S31508000AD02DE9F04115460C460646FFF7EDFE1B4983
S31508000AE0A1FB00377F09A1FB0431480940F2FF3E0C
S31508000AF04FF0010CE046714611E007FB01F300FBDD
S31508000B0005F2B3FBF2F39C0AC3F30903B4F5806F4D
S31508000B1004D29E4502D99E46A44688460139002934
S31508000B20EBD148F4004333617269094B1340013D28
S31508000B3043EA85230CF1FF3C43EA0C43736100202A
S31508000B40BDE8F08101207047012070471F85EB51F1
S31508000B50EF8000FC30B4D0F8084124F0E064C0F817
S31508000B600841D0F80851064C2C4041EA032343EAD1
S31508000B70026244EA0203C0F8083130BC704700BF7D
S31508000B80C0C0FFF830B4D0F80C4124F0E064C0F8D7
S31508000B900C41D0F80C51074C2C4041EA032343EA98
S31508000BA0026244EA020343F08053C0F80C3130BCB9
S31508000BB0704700BFC0C0FFEF10B5144B984208D16C
S31508000BC04FF40060FFF784FE4FF40060FFF768FEFD
S31508000BD010BD0F4B984207D10E4C2046FFF778FE02
S31508000BE02046FFF75DFE10BD0B4B984207D10B4C14
S31508000BF02046FFF76DFE2046FFF752FE10BD40F275
S31508000C004B11074800F0C0FC10BD00BF08000340A8
S31508000C100800024880000010084002480001001041
S31508000C208C1B000810B504462F4B984205D003F5D7
S31508000C300073984203D1012302E0012300E0002358
S31508000C4043B92A4B9C4207D003F500739C4205D151
S31508000C50012304E0012302E0012300E0002343B955
S31508000C60234B9C4207D003F500739C4205D1012310
S31508000C7004E0012302E0012300E000231BB951210F
S31508000C801C4800F081FC184B9C4203D003F5007306
S31508000C909C4203D11848FFF78FFF19E0134B9C427B
S31508000CA003D003F500739C4203D11448FFF784FF71
S31508000CB00EE00F4B9C4203D003F500739C4203D110
S31508000CC00F48FFF779FF03E065210A4800F05CFC4E
S31508000CD00323E360E36813F0010FFBD0236C23F0D2
S31508000CE00F03236410BD00BF000003400000024844
S31508000CF0004002488C1B0008080003400800024810
S31508000D000840024810B5802209210748FFF7ECFD84
S31508000D10064C00220D212046FFF7E6FD236E23F43C
S31508000D200053236610BD00BF00850248008F0248A5
S31508000D3070B586B000238DF80C300126049602257E
S31508000D408DF814500C4C03AA04212046FFF7D8FC52
S31508000D5090238DF8003001968DF808506A460521D3
S31508000D602046FFF7CDFC054AD36923F00703334332
S31508000D70D36106B070BD00BF008102480000034081
S31508000D8008B5FFF7BFFF00F033FCFFF7D1FF00F00F
S31508000D903DFCFCE708B500F03BFA08BD10B500F0CD
S31508000DA0DDFAA0B1FFF794FA88B100F057FC00F01D
S31508000DB0E7FA00F0D7FA20F0604020F07F00044BF5
S31508000DC0186000F0CFFA446800F024FAA04710BD76
S31508000DD008ED00E070B508E0461C4D1C0B78037062
S31508000DE000F06AFC224630462946531E9CB2002A69
S31508000DF0F2D170BD030E082B01D100F18060704757
S31508000E0038B50546002419E000F056FC04EB440208
S31508000E1093000C4AD358AB420ED804EB44018A001F
S31508000E2008490A44526813449D4205D204EB44001B
S31508000E3083000B44187A38BD0134E4B20E2CE3D98A
S31508000E40FF2038BDAC1B000838B50546002410E065
S31508000E5000F032FC04EB44029300084A13441B7A60
S31508000E60AB4204D104EB44018B00D05838BD0134A1
S31508000E70E4B20E2CECD94FF0FF3038BDAC1B00089D
S31508000E8008B5C1F3090353B90368994209D040F874
S31508000E90041B4FF48062FFF79DFF012008BD002068
S31508000EA008BD012008BD00BF2DE9F04106460068CF
S31508000EB0FFF7A6FFFF2833D000272CE000F0FCFB45
S31508000EC035683C0225443444043400F081FA00F1C4
S31508000ED00D0821462846FFF7E1FB05E000F078FA01
S31508000EE0804520D300F0E8FBFFF7D0FB00F00100B7
S31508000EF010F0FF0FF2D1FFF7C9FB30F0100315D140
S31508000F00002305E05A5DD2B2E15C8A4211D1013371
S31508000F10FF2BF7D90137032FD0D90120BDE8F0817F
S31508000F200020BDE8F0810020BDE8F0810020BDE882
S31508000F30F0810020BDE8F08138B50D460B4B98428C
S31508000F4007D004460A4B994205D0FFF7ADFF18B9FA
S31508000F5008E0084C00E0054C29462046FFF790FFBC
S31508000F6010B938BD002038BD204638BDA400002081
S31508000F700040000CA80400202DE9F04106460C4666
S31508000F8017461D4621F47F7828F003080368B3F155
S31508000F90FF3F04D14146FFF773FF034630B333687A
S31508000FA0984505D041463046FFF7C6FF0646D0B1FC
S31508000FB03368E41A3444043400F07EFB331DE31A24
S31508000FC0B3F5806F07D308F580613046FFF7B4FFA5
S31508000FD0064650B1041D17F8013B04F8013B013DD4
S31508000FE0EAD1012302E0002300E000231846BDE809
S31508000FF0F08100BF884230D8F8B505460E4670B372
S315080010000F2926D92DE000F057FB2846FFF71CFFCD
S315080010100746B0F1FF3F26D000F0DAF900F5CE54C6
S3150800102008343846FFF75AFB05E000F0D1F9844248
S315080010301BD300F041FBFFF729FB00F0010010F07D
S31508001040FF0FF2D1FFF722FB30F020030FD1013555
S31508001050EDB2B542D7D90120F8BD0020704700206F
S31508001060F8BD0020F8BD0020F8BD0020F8BD00201E
S31508001070F8BD00BF4FF0FF33024A1360024A1360FF
S31508001080704700BFA8040020A400002070B50D46D4
S315080010901646FFF7AFFE0446FFF7B2FEFF281AD042
S315080010A060190138FFF7ACFEFF2816D024F47F73C9
S315080010B023F003030A4A934206D12B4632462146B9
S315080010C00848FFF759FF70BD2B46324621460648A9
S315080010D0FFF752FF70BD002070BD002070BD00BF35
S315080010E00040000CA4000020A804002070B50C469F
S315080010F0FFF780FE0646FFF783FE054630190138DE
S31508001100FFF77EFEFF2D06D0FF2806D001462846AB
S31508001110FFF770FF70BD002070BD002070BD00BFD6
S31508001120114B1B68B3F1FF3F18D000B583B00E4BC7
S3150800113059689A681144DA6811441A6911445A6957
S3150800114011449A691144DA698B18DB4302AA42F8FA
S31508001150043D04210548FFF799FF01E00120704787
S3150800116003B05DF804FB00BFA40000200042000C99
S315080011700E4B1A6804331B6813440D4A126813444D
S315080011800C4A126813440C4A126813440B4A126834
S3150800119013440B4A12681344DB430A4A1268934203
S315080011A001D1012070470020704700BF0040000CA5
S315080011B00840000C0C40000C1040000C1440000CB9
S315080011C01840000C0042000C08B50D4B1B68B3F123
S315080011D0FF3F04D00A48FFF767FE034668B1094B8C
S315080011E01B68B3F1FF3F05D00648FFF75DFE0346CF
S315080011F010B902E0012300E00123184608BD00BF2C
S31508001200A4000020A8040020004870470040000CF5
S3150800121072B6704762B670470649074A074B9A4244
S31508001220BEBF51F8040B42F8040BF8E704488047A0
S3150800123004480047A41C0008000000206C00002099
S31508001240FD0500085D0200083C493D4A002301E00F
S3150800125041F8043B9142FBD3FFF792FDFEE7FEE718
S31508001260FEE7FEE7FEE7FEE7FEE7FEE7FEE7FEE748
S31508001270FEE7FEE7FEE7FEE7FEE7FEE7FEE7FEE738
S31508001280FEE7FEE7FEE7FEE7FEE7FEE7FEE7FEE728
S31508001290FEE7FEE7FEE7FEE7FEE7FEE7FEE7FEE718
S315080012A0FEE7FEE7FEE7FEE7FEE7FEE7FEE7FEE708
S315080012B0FEE7FEE7FEE7FEE7FEE7FEE7FEE7FEE7F8
S315080012C0FEE7FEE7FEE7FEE7FEE7FEE7FEE7FEE7E8
S315080012D0FEE7FEE7FEE7FEE7FEE7FEE7FEE7FEE7D8
S315080012E0FEE7FEE7FEE7FEE7FEE7FEE7FEE7FEE7C8
S315080012F0FEE7FEE7FEE7FEE7FEE7FEE7FEE7FEE7B8
S31508001300FEE7FEE7FEE7FEE7FEE7FEE7FEE7FEE7A7
S31508001310FEE7FEE7FEE7FEE7FEE7FEE7FEE7FEE797
S31508001320FEE7FEE7FEE7FEE7FEE7FEE7FEE7FEE787
S31508001330FEE7FEE7FEE7FEE7FEE7FEE780000020A1
S315080013409409002008B5FFF795FE08BD08B5FFF714
S315080013509DFE08BD08B5FFF7C9FE08BD08B5FFF72D
S3150800136007FF08BD08B5FFF74FFF08BD08B5FFF72B
S31508001370D7FE034610B1FFF727FF0346184608BDF8
S315080013800022014B1A60704710E000E008B5FFF72D
S31508001390F7FF054B054A5A6000229A600521196035
S315080013A0034B1A6008BD00BF10E000E07F32020060
S315080013B0AC080020044B1B6813F4803F03D0034A93
S315080013C0136801331360704710E000E0AC08002092
S315080013D008B5FFF7EFFF014B186808BDAC080020F9
S315080013E008B50C4BD3F8143113F4805F10D10146BD
S315080013F00848FFF74BFB074BD3F8143113F4807FEB
S31508001400F9D04FF48072034BC3F81821012008BDA8
S31508001410002008BD00000340074BD3F8143113F031
S31508001420080F07D110B504460348FFF741FB2070A3
S31508001430012010BD0020704700000340F0B585B0BC
S315080014404FF46143019308238DF808308DF809306D
S3150800145001258DF80A5010278DF80B700026ADF877
S315080014600C600C4C01A92046FFF7DAFA2B46042239
S3150800147039462046FFF76EFB2B46042231462046A6
S31508001480FFF780FB236C23F00F0343F0020323646A
S3150800149005B0F0BD0000034070B506460D4640296C
S315080014A003D972210F4800F06FF82846FFF798FF16
S315080014B0012803D076210B4800F066F800240CE0DA
S315080014C000F0FAF8305DFFF78BFF012803D07F2183
S315080014D0044800F059F80134A4B2ABB29C42EFD3E9
S315080014E070BD00BF601C000838B5224B1C789CB93B
S315080014F02148FFF791FF01283AD11F4B1B78002B93
S3150800150031D0FFF765FF1D4B186000221C4B1A707F
S315080015100122184B1A702BE00546194B1B7801332C
S3150800152015481844FFF778FF0446012810D1144BD4
S315080015301A780132D2B21A700F4B1B789A4214D11C
S3150800154010492846FFF746FC00220A4B1A700FE09E
S31508001550FFF73EFF094B1B686433984207D90024FE
S31508001560044B1C7004E01C4602E0002400E0002442
S31508001570204638BDF5080020B4080020F8080020E9
S31508001580B0080020B508002008B5024B196000F025
S3150800159093F8FCE7FC08002008B500F085F8012858
S315080015A010D0094B1B78012B0CD1FFF711FF074B05
S315080015B01B6803F5FA73984204D30022024B1A708B
S315080015C0FFF7ECFB08BD00BF000900200409002056
S315080015D008B50122044B1A70FFF7FAFE034B186090
S315080015E0FFF7DAFF08BD00BF000900200409002044
S315080015F008B5FFF7CFFB00F05BF8FFF7C7FEFFF76C
S31508001600A1FE00F00DF8FFF7E3FF08BD08B500F0EE
S3150800161053F8FFF7CFFE00F00FF8FFF7BDFF08BD40
S3150800162008B500F0B5F9FFF709FF0022014B1A705B
S3150800163008BD00BF0000002008B50648FFF754FFA4
S31508001640012805D10022044B1A70024800F0BEF9A1
S3150800165008BD00BF0809002000000020704700BF31
S3150800166008B5044B1B7813B9C9B2FFF715FF00F08C
S31508001670A5F908BD00000020044B1B78013B022B8E
S3150800168001D9402070470020704700BF00000020A5
S31508001690044B1B78013B022B01D9402070470020E0
S315080016A0704700BF0000002008B500F07FF908BDAC
S315080016B008B5FEF71BFE08BD08B5FEF71DFE08BDFA
S315080016C010B4002304E010F8011B0B44DBB22146DA
S315080016D04C1E0029F7D1136001205DF8044B7047B2
S315080016E00022014B5A70704748090020034BFE221E
S315080016F0DA7018710222A3F84420704748090020BE
S3150800170010B5054C00232370FFF7EAFFFF23E370AB
S315080017100123A4F8443010BD48090020064BFF22D7
S31508001720DA7000221A71597859719A71DA711A7237
S315080017300622A3F8442070474809002008B500206F
S31508001740FFF7D4FF08BD00BF084BFF22DA70084A2E
S315080017509A6400221A715A719A710721D9711A72FC
S315080017605A729A720822A3F8442070474809002042
S31508001770881C0008044BFF22DA7042689A6401222A
S31508001780A3F84420704700BF4809002010B5084C4C
S31508001790FF23E370E21D4168A06CFFF791FF2071FB
S315080017A000236371A3710823A4F8443010BD00BF59
S315080017B04809002008B53120FFF798FF08BD00BF8B
S315080017C038B5084CFF23E370002525716571FFF7CE
S315080017D053FFA071E571257265720723A4F844309A
S315080017E038BD00BF4809002038B5FFF779FF0D4C12
S315080017F001252570FF23E3701023237100236371ED
S31508001800FFF73AFFA071FFF743FFE071FFF740FFCC
S31508001810C0F3072020726572A5720823A4F8443025
S3150800182038BD00BF4809002038B505464478FFF79B
S3150800183023FF0138844203DD2220FFF757FF38BD16
S31508001840084C6A78A16C201DFFF7C4FAFF23E370E1
S315080018506B78A26C1344A3646B780133A4F8443004
S3150800186038BD00BF4809002038B504464578FFF75B
S3150800187003FF0138854203DD2220FFF737FF38BD15
S315080018806168084DA9646278281DFFF7A3FAFF234B
S31508001890EB706378AA6C1344AB6463780133A5F8DC
S315080018A0443038BD4809002038B505460D4B9C6CB8
S315080018B0FFF7E2FE6A1C411E2046FFF747FD18B9EE
S315080018C03120FFF713FF38BD064CFF23E370FFF7FF
S315080018D0D3FE0138A36C1844A0640123A4F844304D
S315080018E038BD00BF4809002038B504464578FFF7DB
S315080018F0C3FE0238854203DD2220FFF7F7FE38BD16
S315080019000F4BFF22DA700122A3F84420617831B91F
S31508001910FFF72CFD90B93120FFF7E8FE38BDA21C71
S31508001920074B986CFFF712FD18B93120FFF7DEFE5A
S3150800193038BD6378024A916C0B44936438BD00BF86
S315080019404809002008B54168074B986CFFF702FD67
S3150800195018B93120FFF7CAFE08BD034BFF22DA701B
S315080019600122A3F8442008BD4809002008B5FFF75E
S3150800197015FA034BFF22DA700122A3F8442008BDAA
S315080019804809002008B589B2FFF76AFE08BD00BFFE
S31508001990054B00221A709A6483F84320A3F8442062
S315080019A09A705A70704700BF48090020024B187891
S315080019B000B10120704700BF480900200022024BF1
S315080019C083F84320704700BF4809002008B503780C
S315080019D0FF2B02D1FFF708FF50E0334A1278012A9D
S315080019E060D1C93B352B46D8DFE803F0334545427D
S315080019F045453F363C3945454545454545454545B3
S31508001A004545454545454545454545454545454578
S31508001A10454545454545241E1B2145454527452A37
S31508001A202D30FFF701FF29E0FFF71EFF26E0FFF73D
S31508001A30A1FE23E0FFF7AAFE20E0FFF785FE1DE0E2
S31508001A40FFF77CFE1AE0FFF769FE17E0FFF758FE7E
S31508001A5014E0FFF729FF11E0FFF746FF0EE0FFF756
S31508001A60AFFE0BE0FFF76EFF08E0FFF77FFF05E02C
S31508001A70FFF7A0FE02E02020FFF738FE0A4B93F896
S31508001A804330012B02D11020FFF730FE064BB3F985
S31508001A904410002906DD1846012380F84330033038
S31508001AA0FFF770FF08BD00BF4809002008B5074BBF
S31508001AB0044613B10021AFF30080054B1868836A0A
S31508001AC003B19847204600F033F800BF0000000035
S31508001AD0941C000870B50E4B0E4CE41AA410002591
S31508001AE01E46A54204D056F8253098470135F8E732
S31508001AF000F020F8084C094BE41AA41000251E46ED
S31508001B00A54204D056F8253098470135F8E770BD48
S31508001B1064000020640000206800002064000020A3
S31508001B2002440346934202D003F8011BFAE77047C2
S31508001B30FEE70000F8B500BFF8BC08BC9E46704733
S31508001B40F8B500BFF8BC08BC9E4670472E2E5C6CE4
S31508001B5069625C786D636C69625C7372635C786DEC
S31508001B6063345F6770696F2E630000002E2E5C6C0D
S31508001B7069625C786D636C69625C7372635C786DCC
S31508001B80635F6770696F2E63000000002E2E5C6C21
S31508001B9069625C786D636C69625C7372635C786DAC
S31508001BA0635F757369632E63000000000040000CD4
S31508001BB000400000010000000080000C004000000A
S31508001BC00200000000C0000C0040000003000000F6
S31508001BD00000010C00400000040000000040010C59
S31508001BE000400000050000000080010C00400000D5
S31508001BF00600000000C0010C0040000007000000BD
S31508001C000000020C00000200080000000000040C9E
S31508001C1000000400090000000000080C0000040091
S31508001C200A00000000000C0C000004000B00000075
S31508001C300000100C000004000C0000000000140C4A
S31508001C40000004000D0000000000180C000004004D
S31508001C500E00000000001C0C000004000F0000002D
S31508001C602E2E5C2E2E5C2E2E5C2E2E5C536F7572DD
S31508001C7063655C41524D434D345F584D43345C7542
S31508001C806172742E630000004F70656E424C5400FA
S31108001C90430000000400002000000000D3
S30D08001C9CC0E5FF7F010000000E
S31508001CA4040000000000000000000000000000001E
S31508001CB40000000000000000000000000000000012
S31508001CC400000000901C000800000000000000004E
S31508001CD400000000000000000000000000000000F2
S31508001CE400000000000000000000000000000000E2
S31508001CF400000000000000000000000000000000D2
S31108001D040000000025020008010200088B
S31508001D1000000000000000000000000000000000B5
S30908001D2000000000B1
S70508000000F2
